:020000040000FA
:10000000BD28BA001420200821040319B828B22002
:1000100084133A08800664000D280E28A00A0319EC
:10002000A10F0B288006B828FF3A84178005B8284E
:1000300083178001840AFF3E031D1928B82803177F
:100040008D0083168C130C1483120C08B828031728
:100050008C0083168C130C1555308D00AA308D0042
:100060008C148C1831280C11B828A301A200FF3081
:10007000A207031CA307031CB8280330A100DF302C
:1000800043203728A101E83EA000A109FC30031C51
:100090004C28A00703184928A0076400A10F49288D
:1000A00020185228A01C5628000056280800A1013C
:1000B000A301A20002306928A20003306928A1012F
:1000C000A301A20001306928A20006306928A2001D
:1000D0000530A80023082102031D702822082002F1
:1000E000043003180130031902302805031DFF30C6
:1000F000B8280038031DFF300405031DFF30B82861
:10010000A501A4011030A600210DA40DA50D220803
:10011000A4022308031C230FA50203189628220813
:10012000A40723080318230FA5070310A00DA10D92
:10013000A60B84282008B8281030A800A101A0012F
:10014000A70CA60C031CAA282208A0072308031842
:10015000230FA107A10CA00CA50CA40CA80BA02890
:100160002408B828A009A109A00A0319A10A0800B7
:1001700083130313831264000800831660308F001A
:100180009B013F308500803086008312860120303D
:10019000840060308A011920A030840050308A0128
:1001A00019201030840060308A01182090308400BB
:1001B00060308A01182006160330A300E8308A0157
:1001C00036208A11352903172E308D0003137A0843
:1001D0008A012720640003307A028A11031CF52863
:1001E000F2110330FA028A11F628F215FC016400BC
:1001F00008307C028A1103181A297A08A600A70180
:100200000830A200A3018A019C20B2002508B30097
:100210007C08B2070318B30A32088A011F20B40011
:10022000B5017C083E3E840034088000FC0A8A1137
:10023000031DF72808000130A300F4308A0136209E
:100240000130FC0064007C0874028A11031C34290C
:1002500006167D308A01352006127D308A01352050
:10026000FC0A8A11031D2229080020308400603016
:100270008A011920A030840050308A0119201030E2
:10028000840060308A0118209030840060308A0138
:1002900018200130C6000130C7000130C80001300D
:1002A000C9000130CA000330CB000130CC0003305C
:1002B000CD0006120330A300E8308A013620183042
:1002C0008A011F20D40019308A011F20D5002E304A
:1002D0008A011F20FA008A01E3205408A000550873
:1002E000A100A30100308A0167208A11031D8B2918
:1002F00006160F300505B200B3013208A00033081E
:10030000A100A30101308A0159208A11031D8A2905
:100310008A0179290612640001307A028A11031CCD
:1003200095290230EB008A1197290130EB002F301C
:100330008A011F20E40030308A011F20E500640894
:10034000A6006508A7000530A200A3018A019C2031
:10035000B2002508B3003208A0003308A100043021
:10036000A200A3018A018020D0002108D100E00171
:100370007D30E10007306005D800D90158083E3EC5
:100380008400000886005108A10050088A0143201B
:1003900064008A11051ECE298A11D4296B08E00257
:1003A000031CE1038A01BA295808DE005908DF005E
:1003B0005408A0005508A100A30100308A0167205D
:1003C0008A11031DF9296008003CD4006108031C50
:1003D000013E7D3CD500031718308D0003135408EF
:1003E0008A012720031719308D00031355088A014D
:1003F0002720E001E1011A308A011F20E2001B30B2
:100400008A011F20E3008A113B2533308A011F2017
:10041000E800E901EA01D201D30164008A11051E56
:10042000172AE001E1015808DE005908DF006400E6
:100430008A11F21C1D2A8A11912A64008A11861BD6
:100440004F2A0A308A013520CE0A0319CF0A4E08F6
:10045000A0004F08A1000130A300F4308A016720FA
:100460008A11031D4D2AD201D301EA01E901CE010F
:10047000CF0164008A11F21E3F2A8A010D2A64000E
:100480008A11721F452A8A010D2A64008A11F21905
:100490004D2A06108610061186118A010D2A0A308F
:1004A0008A013520CE01CF010508FB000F30FB0586
:1004B00064008A11861F5E2A8A01582A32308A0116
:1004C00035205208A6005308A7000A30A200A30155
:1004D0008A019C20B2002508B3007B083207D200B5
:1004E00033080318013ED30064006908003C8A11F8
:1004F000031D862AFF307B07B200FF300318013E40
:10050000B3003208463E84000008EA00E90A6400AD
:1005100069086A028A11031D8F2A8A11CB2A8A016F
:100520000D2A0508FB000F30FB0564007B08013C29
:100530008A11031DAC2A0130EF006408A000650891
:10054000A1000530A200A3018A018020D600210865
:10055000D70073108A15502364007B08023C8A116F
:10056000031DC22AEF016408A0006508A100053040
:10057000A200A3018A018020D6002108D7007310B1
:100580008A15502364007B08083C8A11031DC92A80
:10059000F2108A010D2A64008A11721CD12A8A1570
:1005A000452A061664308A013520061264308A0115
:1005B00035205208A0005308A100A30101308A0190
:1005C00067208A11031DD02B64008A11F21EEA2ACB
:1005D0008A11792B64008A11721FF02A8A11A72BC5
:1005E00064007808003C8A11031D322B0030721918
:1005F0000130A00001308A015720B2006808A00035
:1006000000308A015F20B4003208840034088A0177
:100610007920B400B5006400340835048A11031948
:10062000272B6408D6006508D70073100130FD0041
:1006300064007D0868028A11031C272B0130EF003B
:10064000EB018A155023FD0A8A11031D182B013076
:10065000EF00EB01C830D600D70173148A15502380
:100660008A01092A0130EF00EB0164007808013C9F
:100670008A11031D472B6408A6006508A7001930DE
:10068000A200A3018A019C20D6002508D70064009F
:100690007808023C8A11031D592B6408A6006508DE
:1006A000A7000530A200A3018A019C20D6002508DE
:1006B000D70064007808033C8A11031D632B64088B
:1006C000D6006508D700731014308A0135208A15CA
:1006D00050230130EF00EB0164008A11861B722B5E
:1006E0008A01672B0230A30058308A0136208A0124
:1006F000092A0330A300E8308A013620F030A00038
:10070000A1010630840020308A0101200130FD0063
:10071000640006307D028A110318A52B03308A017C
:1007200035200F300505FB00640001307B028A1183
:10073000031CA12B0230A30058308A0136208A0105
:10074000092AFD0A8A11031D882B8A017E2B03309A
:10075000A300E8308A013620F030A000A101063065
:10076000840040308A0101200130FD006400063021
:100770007D028A110318CE2B03308A0135200F30F9
:100780000505FB00640001307B028A11031CCA2BA3
:100790008A01092AFD0A8A11031DB62B8A01AC2B96
:1007A0005208A0005308A100A30102308A0167206B
:1007B0008A11031DC22C64008A11F21EE12B8A11DA
:1007C000702C64008A11721FE72B8A11992C640027
:1007D0007808003C8A11031D292C00307219013061
:1007E000A00000308A015720B2006808A000003045
:1007F0008A015F20B4003208840034088A0179201D
:10080000B400B5006400340835048A1103191E2CA5
:100810006408D6006508D70073100130FD0064003D
:100820007D0868028A11031C1E2CEF010130EB00C9
:100830008A155023FD0A8A11031D0F2CEF01013088
:10084000EB00C830D600D70173148A1550238A01F3
:10085000092AEF010130EB0064007808013C8A119D
:10086000031D3E2C6408A6006508A7001930A200ED
:10087000A3018A019C20D6002508D70064007808CF
:10088000023C8A11031D502C6408A6006508A700CD
:100890000530A200A3018A019C20D6002508D700BC
:1008A00064007808033C8A11031D5A2C6408D600A2
:1008B0006508D700731014308A0135208A1550233B
:1008C000EF010130EB0064008A11861B692C8A015C
:1008D0005E2C0230A30058308A0136208A01092A92
:1008E0000330A300E8308A0136203C30A000A1018B
:1008F0000630840020308A0101200130FD006400B0
:1009000006307D028A110318972C03308A013520A6
:100910000F300505FB00640001307B028A11031CC7
:10092000932C8A01092AFD0A8A11031D7F2C8A0152
:10093000752C0330A300E8308A0136203C30A0003B
:10094000A1010630840040308A0101200130FD0001
:10095000640006307D028A110318C02C03308A011E
:1009600035200F300505FB00640001307B028A1141
:10097000031CBC2C8A01092AFD0A8A11031DA82C1C
:100980008A019E2C5208A0005308A100A301033045
:100990008A0167208A11031DD12C0330F8008A01D7
:1009A000092A5208A0005308A100A30104308A01BB
:1009B00067208A11031DDF2CF8018A01092A5208D9
:1009C000A0005308A100A30105308A0167208A1105
:1009D000031DEE2C0230F8008A01092A5208A000FB
:1009E0005308A100A30107308A0167208A11031D63
:1009F000FD2C0130F8008A01092A5208A000530892
:100A0000A1006430A200A3018A018020B200210865
:100A1000B3003208A0003308A100A30106308A0108
:100A20005920B2005208A0005308A1000A30A200C9
:100A3000A3018A0180202408B4002508B5003408E9
:100A4000A0003508A100A30101308A015920B4009B
:100A50003208840034088A017920B400B5006400AB
:100A6000340835048A110319392D8A113B258A016E
:100A7000092A8A11392E0130F4005208A0005308C7
:100A8000A1000230A30063308A0167208A11031D90
:100A90004B2D0130F4005208A0005308A100023091
:100AA000A3006D308A0167208A11031D592D023081
:100AB000F4005208A0005308A1000230A3007730D0
:100AC0008A0167208A11031D672D0330F400520844
:100AD000A0005308A1000230A30081308A016720E2
:100AE0008A11031D752D0430F4005208A00053082C
:100AF000A1000230A3008B308A0167208A11031DF8
:100B0000832D0530F4005208A0005308A1000230E4
:100B1000A30095308A0167208A11031D912D0630AC
:100B2000F4005208A0005308A1000230A3009F3037
:100B30008A0167208A11031D9F2D0730F400520897
:100B4000A0005308A1000230A300A9308A01672049
:100B50008A11031DAD2D0830F4008A011B210230DB
:100B6000A600A7017408A200A3018A019C20B2007C
:100B70002508B3001830B2070318B30A32088A01F7
:100B80001F20E2000230A600A7017408A200A30102
:100B90008A019C20B2002508B3001930B20703185F
:100BA000B30A32088A011F20E30001306007B20057
:100BB00061080318013EB3006208A0006308A100A9
:100BC0003308A30032088A0167208A11031DEA2D29
:100BD0008A112B2E01306002B2000030031C013E4E
:100BE0006102B3006208A0006308A1003308A300FB
:100BF00032088A0167208A11031D002E8A112B2ECC
:100C00006208A0006308A1006108A30060088A01CF
:100C100067208A11031D102E8A011B21F401080090
:100C20000130EF00EB016208A0006308A100610839
:100C3000A30060088A015C208A11031D222EEF01A7
:100C40000130EB006408D6006508D70073108A15E0
:100C500050238A01D52D640001307A028A11031CC9
:100C6000372E8A011B21F40108008A11392E8A01CE
:100C7000002E5208A0005308A1006430A200A30176
:100C80008A018020B2002108B3003208A000330896
:100C9000A100A30106308A015920B2005208A00029
:100CA0005308A1000A30A200A3018A018020240871
:100CB000B4002508B5003408A0003508A100A30140
:100CC00002308A015920B4003208840034088A01B5
:100CD0007920B400B5006400340835048A11031982
:100CE0002D2F0130F4005208A0005308A10002305B
:100CF000A30064308A0167208A11031D812E013010
:100D0000F4005208A0005308A1000230A3006E3086
:100D10008A0167208A11031D8F2E0230F4005208C9
:100D2000A0005308A1000230A30078308A01672098
:100D30008A11031D9D2E0330F4005208A0005308B1
:100D4000A1000230A30082308A0167208A11031DAE
:100D5000AB2E0430F4005208A0005308A10002306A
:100D6000A3008C308A0167208A11031DB92E05303B
:100D7000F4005208A0005308A1000230A3009630EE
:100D80008A0167208A11031DC72E0630F40052081D
:100D9000A0005308A1000230A300A0308A01672000
:100DA0008A11031DD52E0730F4005208A000530805
:100DB000A1000230A300AA308A0167208A11031D16
:100DC000E32E0830F40006160330A300E8308A0151
:100DD00036200F300505FB0064007B08003C8A11BB
:100DE0000319E92E64007B08023C8A11031D242F9D
:100DF0000230A600A7017408A200A3018A019C206A
:100E0000B2002508B3001830B2070318B30A32083D
:100E100003178D00031360088A0127200230A60003
:100E2000A7017408A200A3018A019C20B200250832
:100E3000B3001930B2070318B30A320803178D0044
:100E4000031361088A0127200612F4010330A3006E
:100E5000E8308A0136208A01092A5208A000530886
:100E6000A1000330A30041308A0167208A11031DCD
:100E7000672F64008A11861B3F2F8A01392F323079
:100E80008A0135200F300505FB00640007307B0226
:100E90008A11031C4D2F8A01092A0130EC006400DD
:100EA0006C087B028A11031C612F0616C8308A0168
:100EB00035200612C8308A013520EC0A8A11031D3C
:100EC0004F2F7B03FA008A01E3208A01092A520886
:100ED000A0005308A1000330A30042308A0167201C
:100EE0008A11031D752F8A0135295208A000530865
:100EF000A1000330A30043308A0167208A11031D3B
:100F0000912F031718308D00003003138A0127201A
:100F1000031719308D00003003138A0127208A013E
:100F200035295208A0005308A1000330A300443023
:100F30008A0167208A15031D2728D201D301E90100
:100F4000F1010230A30058308A0136200F30050528
:100F5000FB0064007B08003C8A11031DC52FCE0AEC
:100F60000319CF0A0A308A0135204E08A0004F0825
:100F7000A1000130A300F4308A0167208A11031D0B
:100F8000C52FCE01CF018A01092A64007B087102B6
:100F90008A11031DCD2F8A01A62F7B08F100640062
:100FA0007B08003C8A1503190728CE01CF01640095
:100FB0007B08083C8A11031DEB2F5208A60053083A
:100FC000A7000830A200A3018A019C20D2002508B6
:100FD000D3008A11FE2F5208A6005308A70008303C
:100FE000A200A3018A019C20B2002508B3007B085F
:100FF0003207D20033080318013ED300E90A640027
:101000006908043C8A15031D07288A1509288A01E6
:10101000A62F5208E4005308E50003172F308D0077
:10102000031364088A012720031730308D0003134F
:1010300065088A012720061664308A0135200612C9
:101040000130A300F4308A0136208A01092A5208AF
:10105000A0005308A1000330A30045308A01672097
:101060008A15031DC5286408DC006508DD005C08DE
:10107000A0005D08A100A2010230A3008A01802027
:10108000F4007408A600A701A2010230A3008A019F
:101090009C20B2002508B3003208DC023308031C90
:1010A000013EDD0264007408003C8A15031D5A28C5
:1010B0000830F4008A011B215C08A0005D08A10033
:1010C0004030A200A3018A018020F4007408A60029
:1010D000A7014030A200A3018A019C20B20025088C
:1010E000B3003208DC023308031C013EDD02640059
:1010F0007408003C8A15031D7F280830F400033073
:10110000A300E8308A0136208A011B215C08A00078
:101110005D08A1000830A200A3018A018020F4002C
:101120007408A600A7010830A200A3018A019C2030
:10113000B2002508B3003208DC023308031C013E6C
:10114000DD0264007408003C8A15031DA9280830DC
:10115000F4000330A300E8308A0136208A011B2105
:101160005C08F40064007408003C8A15031DBA286A
:101170000830F4000330A300E8308A0136208A01E9
:101180001B210130F4008A01092A5208A0005308EB
:10119000A1000330A3004B308A0167208A15031D8C
:1011A000D528F21672138A01092A5208A0005308A2
:1011B000A1000330A3004C308A0167208A15031D6B
:1011C000E528F21272178A01092A5208A000530872
:1011D000A1000330A3004D308A0167208A15031D4A
:1011E000F528F21272138A01092A5208A000530846
:1011F000A1000330A30059308A0167208A15031D1E
:101200000429F2148A01092A5208A0005308A100F7
:101210000330A3005F308A0167208A15031D13295C
:1012200086168A01092A5208A0005308A10003303B
:10123000A30060308A0167208A15031D22298612C7
:101240008A01092A5208A0005308A1000330A30014
:1012500061308A0167208A15031D312906178A012A
:10126000092A5208A0005308A1000330A3006230ED
:101270008A0167208A15031D402906138A01092A5D
:101280005208A0005308A1000330A30069308A016E
:1012900067208A15031DCD29D201D301E901F1018F
:1012A0000230A30058308A0136200F300505FB00BC
:1012B00064007B08003C8A15031D7429CE0A0319BB
:1012C000CF0A0A308A0135204E08A0004F08A1003D
:1012D0000130A300F4308A0167208A15031D7429A8
:1012E000CE01CF018A01092A64007B0871028A15A8
:1012F000031D7C298A1555297B08F10064007B08B1
:10130000003C8A150319B629CE01CF0164007B0881
:10131000083C8A15031D9A295208A6005308A70005
:101320000830A200A3018A019C20D2002508D30026
:101330008A15AD295208A6005308A7000830A2005C
:10134000A3018A019C20B2002508B3007B08320764
:10135000D20033080318013ED300E90A640069088B
:10136000033C8A15031DB6298A15B8298A15552903
:101370005208E800031733308D00031368088A0110
:101380002720061664308A01352006120130A3009A
:10139000F4308A0136208A01092A5208A000530835
:1013A000A1000330A3006A308A0167208A15031D5B
:1013B000452A6808DC00DD015C08A0005D08A1008A
:1013C0004030A200A3018A018020F4007408A60026
:1013D000A7014030A200A3018A019C20B200250889
:1013E000B3003208DC023308031C013EDD02640056
:1013F0007408003C8A15031DFF290830F4000330EF
:10140000A300E8308A0136208A011B215C08A00075
:101410005D08A1000830A200A3018A018020F40029
:101420007408A600A7010830A200A3018A019C202D
:10143000B2002508B3003208DC023308031C013E69
:10144000DD0264007408003C8A15031D292A083057
:10145000F4000330A300E8308A0136208A011B2102
:101460005C08F40064007408003C8A15031D3A2AE5
:101470000830F4000330A300E8308A0136208A01E6
:101480001B210130F4008A01092A5208A0005308E8
:10149000A1000330A3006B308A0167208A15031D69
:1014A0007D2A0616FA308A0135200612FA308A01A2
:1014B00035200616FA308A01352006127214803063
:1014C000ED000330F8006408D6006508D7007310FB
:1014D00072110130FD0064007D086D028A15031C45
:1014E0007A2A0130EF00EB018A155023FD0A8A1594
:1014F000031D6B2A06168A01092A5208A000530808
:10150000A100A30101308A0167208A15031DA22AC8
:1015100006120130FD0064007D086D028A15031C6F
:101520009F2A01307219013AEF0000307219013020
:10153000EB008A155023FD0A8A15031D8B2A061617
:101540008A01092A5208A0005308A100A301023011
:101550008A0167208A15031D4E2B0612030172199A
:101560000130013A03197211031D721564006D08F0
:10157000013C8A15031DF32A0130FD006D08680740
:10158000B200B301B30D7D08A000A1013308A30090
:1015900032088A0161208A15031DDC2A0130721984
:1015A000013AEF00003072190130EB008A15502328
:1015B000FD0A8A15031DBE2A72100130FC0064006A
:1015C0000B307C028A150318F12A061664308A0152
:1015D0003520061264308A013520FC0A8A15031D65
:1015E000DF2A8A01092A64006D08023C8A15031D5E
:1015F000FB2A0130ED0064006D08043C8A15031DD0
:10160000032B0230ED0064006D08083C8A15031DB1
:101610000B2B0430ED0064006D08103C8A15031D8F
:10162000132B0830ED0064006D08203C8A15031D63
:101630001B2B1030ED0064006D08403C8A15031D23
:10164000232B2030ED0064006D08803C8A15031DBB
:101650002B2B4030ED000130FD006D086807B20013
:10166000B301B30D7D08A000A1013308A300320827
:101670008A0161208A15031D4B2B01307219013A32
:10168000EF00003072190130EB008A155023FD0A7B
:101690008A15031D2D2B06168A01092A8A01092A9B
:1016A000640001307A028A15031C682B6F08A600BB
:1016B000A7010230A200A3018A019C20EF006B0861
:1016C000A600A7010230A200A3018A019C20EB0022
:1016D0006B08A000A1016108A30060088A016420D2
:1016E0008A15031D892B0130EC0064000B306C025D
:1016F0008A150318872B061664308A0135200612D6
:1017000064308A013520EC0A8A15031D752B8A0185
:10171000092A6F086007B20061080318013EB30090
:101720003208A0003308A1005508A30054088A011C
:1017300064208A15031DB22B0130EC0064000630D2
:101740006C028A150318B02B061664308A01352006
:10175000061264308A013520EC0A8A15031D9E2B7F
:101760008A01092A640001306F028A15031CBB2B11
:1017700072118A15BC2B72156F086007B2006108E0
:101780000318013EB3006B083202E0003308031C6B
:10179000FF3EE10060085E07B20061080318013EE9
:1017A0005F07B30007303205D80000303305D90099
:1017B000E0300605F00058083E3E84000008B20004
:1017C00032087004860064008A15731CEE2B5708DB
:1017D000A30056088A0136208A15F32B5708A1006A
:0E17E00056088A014320080063008A15F42B86
:02400E006E3F03
:10420000010003000200060004000C000800090081
:104210000100010002000200040004000800080080
:1042200003000300060006000C000C000900090052
:10423000000000000000000000000000000000007E
:10424000000000000000000000000000000000006E
:104250000000000000000000000000000500520007
:084260000D0080008000000049
:00000001FF
